:100000002500C20C02000B0C0600A6058605A40400
:10001000A3056F09A3048809A404780074000606E8
:10002000B402E20A01022E000F028E0003071B0A2F
:100030000E022F000008B302F600F502240AF40CA9
:100040003500F7001802A6010E022F000108310C3E
:100050002400A40510022E00EE0003046E038E029D
:10006000E401A405000228000008A4050A028C008F
:1000700003063C0A0C028A003B00090287003C0090
:10008000A30529091E023C001F023D0009028B0046
:100090003B005C09A3040A028C000306520A1E02FC
:1000A0008A00540A0A02DE012800A404000886041B
:1000B000F40C35000A0C370012090607640A3702EF
:1000C00043075C0A8605010886050008F40C350024
:1000D000060C37006D00A60412090606730A3702E3
:1000E00043076B0A0008AD02A605120906067B0A43
:1000F000000006076B0A37024307750A0008F40C74
:100100003500020C3700120937024307830A000842
:10011000A4051002A40427006B002D00CB090902DE
:10012000A40531002B000E023200E702980A0008F5
:100130001002A4042D00CB090902A40533002B00F2
:100140000E023400E702A50A00081002A4042D00E4
:10015000CB090902A40535002B000E023600E70288
:10016000B20A00081002A4042D00CB090902A4055C
:1001700037002B000E023800E702BF0A0008100209
:10018000A4042D00CB090902A40539002B000E029E
:100190003A00A4040008100C2400FF0C29000902F6
:1001A00080000306DD0A00028B000306DD0A000260
:1001B0002900A40200022E00E400A402A402ED0221
:1001C000CF0A000812090607E90A12092606E50AFD
:1001D000F30A34024306F30A0606F30A86047F098B
:1001E0000606620B74002607F30A61002607F30A6D
:1001F0002606F80A010230004605320CC101310022
:10020000010291014307000B0102C8013100010204
:1002100091014307070B4604320C900027000702A8
:10022000A40591000307170B12022800600B1002AF
:100230002D00ED00070293000307280B110229008F
:1002400012022A0013022B0014022C003509600B45
:10025000ED022C0B2709600B0702950003073A0BF0
:100260001302290014022A0015022B0016022C008A
:100270003509600BED023E0B2709600B0702970062
:1002800003074C0B1502290016022A0017022B0047
:1002900018022C003509600BED02500B2709600B8A
:1002A0000702990003075E0B1702290018022A00B3
:1002B00019022B001A022C003509600B2709600B6C
:1002C000A404E20A86050304A4055003A404A305BC
:1002D0000009A3045709010F4306F60B6609020C37
:1002E0008D000307F60B050C2E000D02AE00030770
:1002F000F60B390003045903A3050009A3045709A9
:10030000010F4306F60B6609010C8D000307F60B7F
:100310000D0299000307F60B0D023A0003045A037D
:10032000A3050009A3048604F40C35003C0C370037
:1003300012090607AD0B37024307A00B8605F60B23
:100340002607980B61002607980B2606A50B0102CD
:100350003000120910022700980B320CA700280C5D
:1003600087000306B60B280C2700BC0BF00C870097
:100370000307BC0BF00C270007023B0086057F0932
:100380008604F40C35003C0C370012090607DC0B20
:1003900037024307CD0B8605F60B2607C50B610018
:1003A0002607C50B46052606D30B0102300046047E
:1003B000120910022800C50B320CA800280C880076
:1003C0000306E50B280C2800EB0BF00C8800030754
:1003D000EB0BF00C280008023C008605A3058909F8
:1003E000A304060CA3051A09A304080A0A0CA30512
:0603F0000D09A304000A40
:100400003700F40C3500B805A3041209A305370220
:100410004307040A7800A60500083700F40C3500ED
:100420009805A3041209A30537024307110A7800AF
:10043000860500083700F40C3500B8059805A304BC
:100440001209A305370243071F0A7800A60586058F
:1004500000087E007F001B0203041C06FE013E0311
:100460003F033C06FE013E033F035C06FE013E03E4
:100470003F037C06FE013E033F039C06FE013E0354
:100480003F03BC06FE013E033F03DC06FE013E03C4
:100490003F03FC06FE013E033F030008080C2E004C
:1004A0007E001C023F001B029F0003075B0A1B0229
:1004B000BF00BE02530A0008100C2E007E007F0011
:1004C00003047D037C037F031B029F0003076B0A69
:1004D0001B02BF0003057E03EE02600A0008000C49
:1004E0002800A809E7076F0A050C890003077A0AA4
:1004F000050C7B0A0902A4053000A404100C24009A
:100500000A0C2D00A30909022000A402ED02820AB0
:100510000008000C280019022900A609E707890A2B
:100520001A022E00EE0003046E038E0228001B0246
:100530002900A609E707970AA8021C022900A609B4
:10054000E7079D0A0008840C2700D30A800CA90A3B
:10055000830C2700A00CC6042A00080C2B00E6041C
:100560006A03C6040306C6050000E605EB02AF0AEF
:100570000000E6040000C605BD0AE605C606E7045D
:10058000E604E707EA0A07020F0EE201CD0AD00AE5
:10059000EA0ACD0AD30AD90AEA0AA7020802AC0A73
:1005A000A7020902AC0AE6050000C605A702A10CD5
:1005B000AB0AC6050000E605080C2B00E60503059E
:1005C000C60703046903E604C605EB02DE0AE60576
:1005D0000000E604C604E605ED0AEE0AC605E707D4
:0405E0000008010806
:021FFE00EA0FE8
:00000001FF
